:020000040000FA
:10000000000083160313880103309F00831203133B
:10001000880141309F0067201020192030200C28D3
:100020000730B000B00B12281F151F1915281E0825
:100030000800B100B201B301B40103146430B1028D
:10004000B20A03181F28B107B20303140A30B10221
:10005000B30A03182728B107B3033108B400080016
:10006000F41080305720F4143030B207B307B407CF
:1000700032085720330857202E3057203408572095
:10008000203057206D305720563057200800F93067
:10009000F0000000F00B49280800F1004720F10BA8
:1000A0004E28080008154720081147200800F500D1
:1000B000F0398800F418881452204720F50E75088E
:1000C000F0398800F4188814522047200800643062
:1000D0004D20F030F40030308800522005304D20A3
:1000E0005220472052200812522028305720083032
:1000F00057200130572006305720803057200C30D1
:04010000572008007C
:02400E00313748
:00000001FF
